:020000040000FA
:0400000069303A2801
:08000800A000030EA100831209
:100010008B1C32288B1031181428B11C3228643004
:10002000010203183128182800001628172818285C
:1000300019281A281B281C281D281E281F283110A3
:10004000B114A810031005190314AA0DA90DA80DC9
:10005000B00B322831152A08AF002908AE00280855
:10006000AD00B11081010B11210E8300A00E200EF6
:02007000090085
:0C007400203084008001840A80300402E7
:10008000031C3C281230B000402283160C3085053A
:1000900087018312850187010730990000309A009B
:1000A000103083168E008312603083168F00831207
:1000B0000030831691009F008312C83083168100A0
:1000C000831231309000003083168C008312103080
:1000D0008B00BC1B7128851971286400851D6D2853
:1000E000DC233C1C74283D2381018E018F010B1100
:1000F0008B100B108C018B178C203119A22022221F
:10010000B30B8A28031085190314B90DF030390296
:100110000319A3214E237C286400311808000B1D0D
:1001200008000B11B11031141230B000051D9D28CC
:10013000321483160113831208003210831601173C
:100140008312080031110130B70085144008013EC8
:10015000CE000F08CF008B132030370783169B008B
:100160001C141A088312A400A500C030A506103084
:10017000370783169B001C141A088312A300003053
:10018000370783169B001C141A088312A2008B17D2
:10019000321CD02822090339A200A309A409A50909
:1001A00022082D02031D9D2923082E02031D9D29CF
:1001B00024082F02031D3A2901303702031DE728C6
:1001C0003C19E6283D18E7283D143E145D22023014
:1001D0003702031DF2283C19F128BD18F228BD147E
:1001E0003E146A2203303702031DFD283C19FC2807
:1001F0003D19FD283D153E14772204303702031DBA
:1002000008293C190729BD190829BD153E14842267
:1002100005303702031D13293C1912293D1A1329F1
:100220003D163E14912206303702031D1E293C194B
:100230001D29BD1A1E29BD163E149E220730370205
:10024000031D29293C1928293D1B29293D173E1446
:10025000AB2208303702031D34293C193329BD1B5A
:100260003429BD173E14B82209303702031D3A293C
:100270003E14C52225082F02031D9D290130370297
:10028000031D49293C1948293D1C49293D103E14AC
:10029000EC2202303702031D54293C195329BD1C9E
:1002A0005429BD103E14F02203303702031D5F298C
:1002B0003C195E293D1D5F293D113E14F422043096
:1002C0003702031D6A293C196929BD1D6A29BD1120
:1002D0003E14F82205303702031D75293C19742994
:1002E0003D1E75293D123E14FC2206303702031DC7
:1002F00080293C197F29BD1E8029BD123E14002390
:1003000007303702031D8B293C198A293D1F8B2991
:100310003D133E14042308303702031D96293C196F
:100320009529BD1F9629BD133E14082309303702B5
:10033000031D9C293E140C239D29B70A0A3037025D
:1003400003180800AB280130B600B300B400B500B4
:10035000B70085018701B1138C20B30BE929031085
:1003600085190314B90DF03039020319102AB41F8E
:100370008510B40BE929013037020319102302302C
:1003800037020319142303303702031918230430EA
:10039000370203191C2305303702031920230630C6
:1003A00037020319242307303702031928230830A2
:1003B000370203192C230930370203193023370879
:1003C000B6080319B6000319E7298514B603963059
:1003D000B400311DAC293111321CF3292D09033928
:1003E000AD00AE09AF092F1CB1132F1CAC29B11BF6
:1003F000AC292E18AC29B1178B1320303707BB005E
:100400002F08BA002B2210303707BB002E08BA0085
:100410002B2200303707BB002D08BA002B228B1788
:1004200085018701083037022030031985002A3002
:1004300003198700B70AB6010A303702031CAC293A
:100440003D2308003E1C08003E101030BB003D0854
:10045000BA002B2208008B133A0883161C159A0049
:1004600083123B0883169B0055309D00AA309D00E7
:100470009C1464009C18392A1C1183128B170800E5
:10048000831600309B001C141A088312BC008316CC
:1004900010309B001C141A0883123C18BD008316F0
:1004A00020309B001C141A088312C1000130C11BAC
:1004B000C100C1080319C10008003C198716400893
:1004C0003C1D40034107D0000F08D100BC19372361
:1004D0003D1408003C19071640083C1D4003410725
:1004E000D2000F08D300BC193723BD1408003C19F3
:1004F000871540083C1D40034107D4000F08D50074
:10050000BC1937233D1508003C19051640083C1D51
:1005100040034107D6000F08D700BC193723BD158B
:1005200008003C19851640083C1D40034107D800CF
:100530000F08D900BC1937233D1608003C190715D0
:1005400040083C1D40034107DA000F08DB00BC19DE
:100550003723BD1608003C19871440083C1D400392
:100560004107DC000F08DD00BC1937233D170800E8
:100570003C19071440083C1D40034107DE000F08EA
:10058000DF00BC193723BD170800BC1908003C1D4B
:10059000CD2A303085043F3087048E018F01C001A1
:1005A000D001D201D401D6010130D800DA00DC003C
:1005B000DE004030D1008030D300C030D500FF30A5
:1005C000D7004030D9008030DB00C030DD00FF3084
:1005D000DF00FF30BD00080087128E018F01080088
:1005E00007128E018F01080087118E018F0108000C
:1005F00005128E018F01080085128E018F010800FF
:1006000007118E018F01080087108E018F010800ED
:1006100007108E018F01080037238E018F0108001B
:100620000708203A870008000708103A87000800EA
:100630000708083A870008000508103A85000800F6
:100640000508203A850008000708043A87000800DA
:100650000708023A870008000708013A87000800E7
:100660000508303A850007083F3A87000800CF3078
:100670008505C0308705BD0108003D188716BD18E7
:1006800007163D198715BD1905163D1A8516BD1AA1
:1006900007153D1B8714BD1B071408003C19522B7E
:1006A0003D1C5E2B50084002031D5E2B51080F02BB
:1006B000031C5E2B3C1987123C1D87163C19622BCC
:1006C000BD1C6E2B52084002031D6E2B53080F02F7
:1006D000031C6E2B3C1907123C1D07163C19722B8C
:1006E0003D1D7E2B54084002031D7E2B55080F0232
:1006F000031C7E2B3C1987113C1D87153C19822B4E
:10070000BD1D8E2B56084002031D8E2B57080F026D
:10071000031C8E2B3C1905123C1D05163C19922B0F
:100720003D1E9E2B58084002031D9E2B59080F02A8
:10073000031C9E2B3C1985123C1D85163C19A22BCF
:10074000BD1EAE2B5A084002031DAE2B5B080F02E4
:10075000031CAE2B3C1907113C1D07153C19B22B8D
:100760003D1FBE2B5C084002031DBE2B5D080F021F
:10077000031CBE2B3C1987103C1D87143C19C22B4F
:10078000BD1FCE2B5E084002031DCE2B5F080F025B
:10079000031CCE2B3C1907103C1D07144E084002C9
:1007A000031DD72B4F080F02031CD72B85100C1CE1
:1007B00008000C10C00A0800B601B301B4013C1CCB
:1007C000E42BBC01BC14F02BBC1CE92BBC013C1578
:1007D000F02B3C1DEE2BBC01BC15F02BBC013C14D6
:1007E0003C08B6006400F42BF52BF62BF72BF82B06
:1007F000B41B8716B41F8712B30BF22BB40BF22B6A
:100800000310B60CB608031DF22B0030BB003C08E9
:06081000BA002B220800D3
:084000000800030006000600A1
:02400E00CC33B1
:10420000010003000300030003000200020002009B
:1042100002000000000000000000FF00FF00FF009F
:10422000000000000000000000000000000000008E
:104230000000C000C000C000C000FF00FF00FF0081
:104240000100C300F300CF00FF00C300F300CF0064
:10425000FF00C300F300CF00FF00FF00FF00FF00DE
:10426000FF00FF00FF00FF00FF00FF00FF00FF0056
:10427000FF00FF00FF00FF00FF00FF00FF00FF0046
:10428000FF00FF00FF00FF00FF00FF00FF00FF0036
:10429000FF00FF00FF00FF00FF00FF00FF00FF0026
:1042A000FF00FF00FF00FF00FF00FF00FF00FF0016
:1042B000FF00FF00FF00FF00FF00FF00FF00FF0006
:1042C000FF00FF00FF00FF00FF00FF00FF00FF00F6
:1042D000FF00FF00FF00FF00FF00FF00FF00FF00E6
:1042E000FF00FF00FF00FF00FF00FF00FF00FF00D6
:1042F000FF00FF00FF00FF00FF00FF00FF00AA001B
:00000001FF
